:020000020000FC
:0200000006C038
:10000C0037C200E10ABB0FEE0BBB0FED0DBF6FEF5C
:10001C0006B301FD662700E00ABB0FEF0BBB05E042
:10002C0007BB02E008BB00E808B900E205BF03E02B
:10003C0000B900E000BF00E003BF0FEF06BF00E017
:10004C000FBD0AE00EBD01E00BBD0FE90ABD02E0D9
:10005C000CB933275527FF248827992771E041E0F5
:10006C0006B301FF662700E10ABB0FEE0BBBA7D05E
:10007C0006B301FD662700E00ABB0FEF0BBB7894BB
:10008C008895FECF00916000003019F00A9500931E
:10009C00600009B307FB0F70423071F04330C1F0C0
:1000AC001091620000936200F0F820E02ABB2FEB65
:1000BC002BBB20E42ABB17C0109163000093630094
:1000CC00F1F820E02ABB2FEE2BBB20E12ABB0BC0A2
:1000DC001091640000936400F2F820E02ABB2FED2D
:1000EC002BBB20E22ABB21E0101729F010916000F5
:1000FC00103009F420E0209365001EE12FE002137C
:10010C00109360000F3029F010916100139510933B
:10011C00610010916000103019F410E01093610030
:10012C00109161001A3A41F410E01093610007300D
:10013C0019F4433009F4FFC020916500203009F018
:10014C002AC0423079F04330D1F00E3009F47FC030
:10015C000D3009F488C00B3009F491C0073009F454
:10016C009EC019C00E3009F476C00D3009F47FC062
:10017C000B3009F488C0073009F48DC00CC00E3068
:10018C0009F46DC00D3009F476C00B3009F47FC052
:10019C00073009F49CC00895333019F020E015E8BD
:1001AC0002C020E015EAE117F20720F401931FEFDB
:1001BC00108304C0DCD0CAD0DAD0C8D00895F0E0E7
:1001CC00E6E60FEF008308955527E199FECFF0E0A6
:1001DC00E6E622272EBBE09A1DB301912395011769
:1001EC0021F40A30B8F35FEF08C0C1D0AFD0BFD054
:1001FC00ADD0BDD0ABD0BBD0A9D00895F0E0E6E631
:10020C0010A101910117B9F40A30D0F3F0E0E6E641
:10021C002227E199FECF2EBBE09A0DB31191011765
:10022C0021F02EBB1DBBE29AE19A23951A3088F37C
:10023C006627C2D009C09BD089D099D087D097D0DF
:10024C0085D095D083D093D03327C298089501E000
:10025C00A3DF8DD0089502E09FDF89D0089503E0DD
:10026C009BDF85D0089504E097DF81D0089505E0E9
:10027C0093DF7DD0089506E08FDF79D0089507E0F5
:10028C008BDF75D0089508E087DF71D0089509E001
:10029C0083DF6DD0089500E07FDF69D00895882753
:1002AC009927C298303019F0332789DF0EC028B354
:1002BC00713019F489DF28B350FDC09880DF20FF1E
:1002CC0004C0C09902C08DD001C051D00895313006
:1002DC0099F0323001F1333059F176DF28B350FD0B
:1002EC00C09A6DDF50FD9BD05F3F21F420FD02C012
:1002FC0087D001C03CD01EC067DF61DF3327C298B6
:10030C005F3F39F432E0C29A43D020D01FD040D0A6
:10031C0011C02DD00FC0F0E0E6E80FEF008333E002
:10032C0037D014D013D034D011D010D031D002C06B
:10033C0065DF45DF089543DFC29A31E06F3F21F45A
:10034C0032E026D003D002D023D0089510E500E08F
:10035C000A95F1F71A95E1F7089521E010E000E015
:10036C000A95F1F71A95E1F72A95D1F7089502E469
:10037C0000BF02E003BF02E306BF10E100E00A95F4
:10038C00F1F71A95E1F700E000BF00E003BF089514
:10039C0002E400BF02E003BF02E306BF22E010E864
:1003AC0000E00A95F1F71A95E1F72A95D1F700E0EC
:1003BC0000BF00E003BF089502E400BF02E003BFEA
:1003CC0000E506BFCADF01E406BFC7DF02E306BFD4
:1003DC00C4DF03E206BFC1DF00E000BF00E003BFE3
:1003EC00089502E400BF02E003BF0DE206BFAEDFDA
:1003FC0006E406BFABDF00E000BF00E003BF0895DA
:10040C0002E400BF02E003BF06E406BF9FDF0DE27B
:10041C0006BF9CDF00E000BF00E003BF0895723010
:10042C0029F0733031F0743039F0089591E088EC94
:10043C00089593E088E5089598E088E008950F2DDD
:10044C00F2940F1509F008950770073039F0063053
:10045C0049F0053049F0033049F002C070E00895CE
:10046C0071E0089572E0089573E0089574E00895C2
:10047C0009DE4A9571F443E0E2DF002780309007F3
:10048C0029F08A9531F49A9521F4ABDF723008F09B
:04049C00C098189557
:00000001FF
